:100000003BC0CCC154C053C052C051C050C04FC0FF
:100010004EC04DC04CC04BC04AC049C048C047C08C
:1000200046C045C044C0040309041C0377007700A0
:1000300077002E00660069007300630068006C00A2
:100040002E00640065000E0355005300420061005D
:100050007300700012011001FF000008C016DC05DB
:1000600002010102000109021200010100801909C8
:10007000040000000000000011241FBECFE5D4E002
:10008000DEBFCDBF10E0A0E6B0E0E4E8FEE002C0D5
:1000900005900D92A236B107D9F710E0A2E6B0E0C4
:1000A00001C01D92A33AB107E1F7AED4EAC6A8CFCA
:1000B00085B7836085BF8BB780648BBF08950F932E
:1000C0001F93CF93DF9360918700161604F563505A
:1000D00080918400C7E9D0E0C81BD10980918300DA
:1000E0008D3209F44BC08091620087FD4CC0CE0177
:1000F0009ED48F3F09F483C0882309F458C020E0C0
:1001000030E030936200209360001092870080916D
:10011000610084FF27C0809160008F3F19F1682F34
:100120008930E0F5861B809360008091620080FD3D
:1001300033C00BE48F5F8093620087FD68C0662345
:1001400009F454C088E790E013D5682F162F693062
:1001500008F479C08FEF809360009EE100937700F0
:10016000909361009AE086B3837009F0F5C09150D6
:10017000D1F71092880010928200EEC08AE5809339
:1001800061006830B9F020E030E8309362002093DD
:10019000600010928700BBCF03ECCCCF68E0861BD9
:1001A000809360008091620080FFC3CFF5CF2FEF76
:1001B00030E0EBCF8881807609F05AC020E830E04B
:1001C000109280008981882309F059C01092810023
:1001D000309386002093850022E030E88F818823C9
:1001E000A1F68E81821788F6282FCFCF60E088E7AE
:1001F00090E0D0D094E08FEF80936000AFCF8093F9
:1002000060008EE1809361002FEF30E07ACF209183
:1002100085003091860086FF1EC0462F41504F3F1B
:1002200069F0F901942FA8E7B0E084918D9331969D
:100230009150D8F72F5F3F4F240F311D3093860028
:100240002093850083CF88E790E0A4D0912F9C5F16
:10025000183089F683CF462F41504F3F79F3F9018B
:10026000942FA8E7B0E081918D939150E0F7E2CF11
:10027000CE01CCD4282F8F3FA9F030E8AFCF853006
:1002800059F08630A9F08830E9F0893021F18A30C0
:1002900041F120E030E8A2CF8A818093880020E0FD
:1002A00030E89CCF888187FF2BCF2E8130E029CF8B
:1002B0008B818130E9F0823081F1833011F120E0CF
:1002C00030EC8CCF8AE890E0909386008093850094
:1002D00021E030E883CF8A8180938A0020E030E8F3
:1002E0007DCF309386002093850021E030E876CFE3
:1002F00084E590E0909386008093850022E130ECC5
:100300006DCF8A81882391F486E290E090938600F5
:100310008093850024E030EC61CF86E690E09093F6
:1003200086008093850022E130EC58CF813059F06F
:10033000823029F686E490E09093860080938500D1
:100340002EE030EC4BCF8AE290E0909386008093D1
:1003500085002CE130EC42CFDF91CF911F910F91BE
:100360000895A82FB92F8FEF9FEF41E050EA615019
:1003700070F02D9138E0722F782796958795269505
:1003800070FF02C0842795273A95A9F7F0CF809592
:1003900090950895E6DF8D939D930895CF93CFB701
:1003A000CF93B09BFECFB09B09C0B09B07C0B09B62
:1003B00005C0B09B03C0B09B01C09EC0DF93C0913D
:1003C0008400DD27C557DF4FB09B02C0DF91EBCF24
:1003D0002F930F931F9306B32FEF00FB20F94F933A
:1003E0003F9316B34FEF012700FB21F93BE031C0EB
:1003F0004E7F012F16B3216028C0102F4D7F226041
:10040000000006B329C04B7F2460012F000016B303
:100410002BC016B3477F28602AC04F7E06B32061E9
:100420002CC04F7D16B320622FC04F7B06B32064D3
:1004300032C0422706B349934FEF0000102710FB4C
:1004400020F916B31370A9F1297F91F2012700FB5F
:1004500021F906B3237F89F23150F0F1102710FB08
:1004600022F916B3277E79F2012700FB23F92F7CAE
:1004700081F206B3102710FB24F92F7971F200C026
:1004800016B3012700FB25F92F7359F200C006B3FC
:10049000102710FB26F9223040F200C016B30127C6
:1004A00000FB27F9243028F64F77206816B30000A8
:1004B000F9CF3B503195333010E41ABFB8F0C31B6D
:1004C000D0400881033C41F10B3431F11981412FB7
:1004D0001F7720918200121731F4093691F10D3205
:1004E00079F0013E69F02227209389003F914F91D6
:1004F0001F910F912F91DF91CF91CFBFCF91189581
:10050000009389003F914F911F910F912F91DF919F
:10051000CAB7C6FD46CFF0CF00918900002331F362
:1005200010918700112349F534304AF13093870048
:1005300000938300109184003BE0311B30938400D2
:100540001EC0009187000130C4F40AE530916100BB
:1005500034FD17C000936100C7E7D0E016C005273F
:1005600010E008BB1FC0052722C0052727C00527AC
:100570002CC0052710E008BB33C04AE503C042ED9C
:1005800001C0432FC4E1D0E032E017B31360C09A3A
:1005900008B317BB5F9353E020E820FF052708BB93
:1005A000279517951C3FD8F620FF0527279508BBF0
:1005B00017951C3FC0F620FF05272795179508BB08
:1005C0001C3F98F620FF0527279517951C3F08BB71
:1005D00070F600C0499120FF052708BB27951795A5
:1005E0001C3F38F620FF0527279508BB17951C3FB1
:1005F00038F520FF05272795179508BB1C3F10F5F8
:1006000020FF0527279517951C3F08BBE8F4242FEA
:100610003A9519F60C7F5F9108BB00C010918800D5
:10062000C651D04011F01093820010E41ABF01604F
:1006300017B31C7F402F4C7F08BB17BB48BB56CF5E
:100640000527D3CF0527D8CF0527DDCFA398AB9AB1
:10065000000000009B9904C082E58DB91EB8089582
:10066000A29AAA98000000009B9B07C082E58DB962
:1006700081E08EB9A298AA9A089583E58DB91EB833
:10068000A298AA9A0895882339F488E793E0909372
:10069000A2008093A100089585E993E09093A200C1
:1006A0008093A100089592B782B7891B8C30E0F344
:1006B0000895C49AA59AAD9887B38C6287BBC298F7
:1006C000C598F1DFC29AEFDFC2988091A1009091A6
:1006D000A2008559934009F00895B8DF089587B3C3
:1006E000837D87BB88B3837D88BBA5981DB808959B
:1006F000FF920F931F93182FFF2400E00CC0C398A4
:10070000FF0CB499F394CFDFC59ACDDFC5980F5F86
:10071000083029F0110F17FFF2CFC39AF1CF8F2DB8
:1007200090E01F910F91FF9008958FB9779BFECFB6
:100730008FB190E008950F931F930FE103C0015014
:100740000F3F51F1E091A100F091A2008CEA0995D0
:10075000E091A100F091A20083E50995E091A1004C
:10076000F091A20080E00995182FE091A100F0918E
:10077000A20080E00995133591F01DB8C59A93DF6A
:10078000C59891DF8091A1009091A2008559934076
:10079000B1F65CDF0150B0F681E090E002C080E08D
:1007A00090E01F910F910895EF92FF920F931F9386
:1007B0007B018C01862F8170880F880F880FE09154
:1007C000A100F091A20080620995D801C70129E03B
:1007D000B695A795979587952A95D1F7E091A100B1
:1007E000F091A200099516950795F794E794E0918A
:1007F000A100F091A2008E2D0995E091A100F09149
:10080000A20080E0099590E01F910F91FF90EF907A
:1008100008950F931F938C01E091A100F091A20025
:1008200080EA0995812F9927E091A100F091A2001B
:100830000995E091A100F091A200802F0995E09127
:10084000A100F091A20080E0099590E01F910F9126
:100850000895FF920F931F938C01F62EE091A10053
:10086000F091A20080EC0995812F9927E091A100D9
:10087000F091A2000995E091A100F091A200802FD3
:100880000995E091A100F091A2008F2D09958EE1CC
:10089000AED080E090E01F910F91FF900895CF922D
:1008A000DF92EF92FF920F931F936B017C01142F45
:1008B000E091A100F091A2008CE40995E091A100E3
:1008C000F091A200D701C60169E0B695A79597956A
:1008D00087956A95D1F70995E091A100F091A20062
:1008E000D701C601B695A795979587950995E0918B
:1008F000A100F091A20080E009951F3FA9F002B786
:100900001EE1C701B60150DF8F3F59F482B7801B4B
:100910008D3310F002B71150112399F781E090E068
:1009200007C080E090E004C08FE061D080E090E0FC
:100930001F910F91FF90EF90DF90CF900895CF928D
:10094000DF92EF92FF920F931F936B017C01042FB4
:10095000122FE091A100F091A200862F8170880FE4
:10096000880F880F80640995E091A100F091A200A2
:10097000D701C60129E0B695A795979587952A9541
:10098000D1F70995E091A100F091A200D701C6012D
:10099000B695A795979587950995E091A100F09157
:1009A000A200802F09951123A1F00F37A9F002B7FB
:1009B0001EE1C701B601F8DE8F3759F482B7801BFC
:1009C0008D3310F002B71150112399F781E090E0B8
:1009D00007C080E090E004C08FE009D080E090E0A4
:1009E0001F910F91FF90EF90DF90CF900895382FD7
:1009F000882349F020E092B782B7891B8C33E0F35B
:100A00002F5F2317C1F7089512BA18BA8BEF81BB75
:100A10008FEF87BB17BA93E094BB8EEF85BB93BF74
:100A200081E031DE45DB78944ADB49DBFDCFFF9284
:100A30000F931F93CF93DF93062F209163002130F4
:100A400029F0243019F08FEF90E08CC0002309F4D6
:100A500087C0EC01FF2410E051C080917300909199
:100A60007400892B09F057C060916F00709170007D
:100A70008091710090917200488161DF80916400E3
:100A80009091650001979093650080936400892B95
:100A9000E1F4109263008091750081FF39C080916C
:100AA000760090E0209173003091740082179307D4
:100AB00079F160916F007091700080917100909158
:100AC00072004881ECDEFF24F39480916F009091D6
:100AD0007000A0917100B09172000196A11DB11D2E
:100AE00080936F0090937000A0937100B093720098
:100AF0001F5F2196101789F120916300213009F4BE
:100B0000ACCF688180916F0090917000A2DEB6CF6B
:100B1000FF24F394DACF60916F00709170008091A0
:100B200071009091720020E0488109DF8091760089
:100B3000815080937600882309F0A0CF60916F00E8
:100B40007091700080917100909172004881A7DED1
:100B5000809173008093760091CF8F2D90E002C03A
:100B600080E090E0DF91CF911F910F91FF90089569
:100B70000F931F93CF93DF93AC01062F2091630057
:100B8000822F8250823018F08FEF90E03AC06623B7
:100B9000A1F1EA0110E01FC080916F0090917000F8
:100BA00038DE888380916F0090917000A091710071
:100BB000B09172000196A11DB11D80936F009093BA
:100BC0007000A0937100B09372001F5F2196101700
:100BD00079F0209163002230F9F660916F007091F6
:100BE00070008091710090917200DEDD8883DACF11
:100BF000083018F0802F90E004C010926300802F1E
:100C000090E0DF91CF911F910F910895CF93DF93E3
:100C1000EC018981813041F1823009F4CBC083300D
:100C200009F4CDC0843059F1873009F499C085307A
:100C300009F418C1863009F44FC0883009F4E2C0C5
:100C4000893079F481E0809366008A819B81AC8150
:100C5000BD8180936F0090937000A0937100B0935A
:100C6000720020E030E003C19A9933C080E00BDDD0
:100C700010926600A9981DDD20E030E0F8C0809158
:100C800066008823A1F48B8190E0982F88272A8121
:100C900030E0822B932BAA2797FDA095BA2F809343
:100CA0006F0090937000A0937100B09372008F81D9
:100CB00090E0982F88272E8130E0822B932B909301
:100CC00065008093640082E0809363002FEF30E042
:100CD000CEC081E0D8DCCCCF809166008823A1F41F
:100CE0008B8190E0982F88272A8130E0822B932BEC
:100CF000AA2797FDA095BA2F80936F00909370005C
:100D0000A0937100B09372008C819D81292F2F7068
:100D100020937500492F50E0407F507042955295C6
:100D2000507F5427407F5427480F511D5093740023
:100D30004093730020FF02C0409376008F8190E0C3
:100D4000982F88272E8130E0822B932B909365007B
:100D50008093640081E0809363002FEF30E087C0D0
:100D6000809166008823A1F48B8190E0982F8827DA
:100D70002A8130E0822B932BAA2797FDA095BA2FCA
:100D800080936F0090937000A0937100B0937200F5
:100D90008F8190E0982F88272E8130E0822B932B33
:100DA000909365008093640083E0809363002FEF4D
:100DB00030E05DC094DCA99A20E030E058C0E091BA
:100DC000A100F091A2008A81099580936700E091CB
:100DD000A100F091A2008B81099580936800E091B9
:100DE000A100F091A2008C81099580936900E091A7
:100DF000A100F091A2008D81099580936A0024E002
:100E000030E035C0809166008823A1F48B8190E0AA
:100E1000982F88272A8130E0822B932BAA2797FDD1
:100E2000A095BA2F80936F0090937000A0937100EB
:100E3000B0937200109274001092730010927500BB
:100E40008F8190E0982F88272E8130E0822B932B82
:100E5000909365008093640084E0809363002FEF9B
:100E600030E005C068DC8093670021E030E087E671
:100E700090E09093860080938500C901DF91CF9127
:040E80000895FFCF03
:020E8400FF5A13
:00000001FF
